:1000000024C10000AFC7000082C7000055C7000030
:1000100028C70000FBC60000CEC6000047C1000094
:1000200045C1000043C1000041C100003FC10000C4
:100030003DC100003BC1000039C1000037C10000D4
:1000400035C1000033C1000031C100002FC10000E4
:100050002DC100002BC1000029C1000062C60000B4
:1000600025C1000028C60000FDC500001FC100001A
:100070001DC100001BC1000019C1000017C1000014
:1000800015C1000013C1000011C100000FC1000024
:100090000DC100000BC1000009C1000007C1000034
:1000A00005C1000003C1000001C10000FFC0000045
:1000B000FDC00000FBC00000F9C00000F7C0000058
:1000C000F5C00000F3C00000F1C00000EFC0000068
:1000D000EDC00000EBC00000E9C00000E7C0000078
:1000E000E5C0000000002100240027002A002D00A8
:1000F0003000330001010000040107010A01000083
:100100002200250028002B002E00310034000201BF
:100110000000050108010B0100002000230026005B
:1001200029002C002F00320000010000030106010D
:10013000090105050505070508080808020202026D
:100140000A0A080804040404010101010101010173
:100150000303030303030303040707070C0C0C0C3E
:100160000C0C0C0C02020202060606060606060627
:100170000B0B0B0B0B0B0B0B0102102020080810B4
:100180002040102040800201020108040201010207
:1001900004081020408080402010080402018004E0
:1001A000020180402010080402010804020101023B
:1001B0000408102040800102040810204080000044
:1001C0000A0B02090C0D0E080703040100000000D1
:1001D000000000000000000000000000000000001F
:1001E00000000000000000000000121110000000DC
:1001F00000000000000000000000000000000000FF
:10020000000000003D300A003D310A000A003D3088
:100210000A002E4F46460A003D310A002E4F4E0A74
:10022000003D300A003D310A000A000A000A00239E
:100230000023002300232323235265616C53696D3F
:10024000476561722300AC08F10E11241FBECFEF89
:10025000D1E2DEBFCDBF00E00CBF2AE0A2E5B6E0F0
:1002600001C01D92AD38B207E1F716E0A0E0B2E0A0
:10027000E8E5F3E200E00BBF02C007900D92A23563
:10028000B107D9F711E0C4E2D1E000E006C0219740
:100290000109802FFE010E945C0FC332D10780E06C
:1002A0000807A9F70E94AA090C949B11A9CEAF9246
:1002B000BF92CF92DF92EF92FF920F931F93CF9353
:1002C000DF936C017B018B01040F151FEB015E01B5
:1002D000AE18BF08C017D10759F06991D601ED914A
:1002E000FC910190F081E02DC6011995892B79F7D9
:1002F000C501DF91CF911F910F91FF90EF90DF909B
:10030000CF90BF90AF900895FC01538D448D252F61
:1003100030E0842F90E0821B930B541710F0CF969F
:10032000089501970895FC01918D828D981761F0D1
:10033000A28DAE0FBF2FB11D5D968C91928D9F5FE8
:100340009F73928F90E008958FEF9FEF0895FC01C7
:10035000918D828D981731F0828DE80FF11D858D7A
:1003600090E008958FEF9FEF0895FC01918D228D0D
:10037000892F90E0805C9F4F821B91098F73992792
:1003800008958BEF96E0F1DF21E0892B09F420E05E
:10039000822F0895FC01A48DA80FB92FB11DA35A77
:1003A000BF4F2C91848D90E001968F739927848F95
:1003B000A689B7892C93A089B1898C9183708064B8
:1003C0008C93938D848D981306C00288F389E02D59
:1003D00080818F7D80830895EF92FF920F931F930A
:1003E000CF93DF93EC0181E0888F9B8D8C8D9813E8
:1003F0001AC0E889F989808185FF15C09FB7F894F4
:10040000EE89FF896083E889F9898081837080643F
:1004100080839FBF81E090E0DF91CF911F910F918A
:10042000FF90EF900895F62E0B8D10E00F5F1F4F99
:100430000F731127E02E8C8D8E110BC00FB607FCA9
:10044000FACFE889F989808185FFF5CFCE01A2DF57
:10045000F2CFEB8DEC0FFD2FF11DE35AFF4FF08231
:100460009FB7F8940B8FEA89FB8980818062D0CF97
:100470000F931F93CF93DF938C01D0E0C0E0F8017E
:10048000EC0FFD1F6491662339F08BEF96E0A4DF3B
:10049000892B11F02196F3CFCE01DF91CF911F91DF
:1004A0000F910895CF93DF93EC01888D8823B1F0ED
:1004B000AA89BB89E889F9898C9185FD03C080816F
:1004C00086FD0CC00FB607FCF7CF8C9185FFF2CFED
:1004D000808185FFEDCFCE015DDFEACFDF91CF9147
:1004E00008958150823108F05AC0E82FF0E0882743
:1004F000E358FD4F8F4F0C945C0F9D02A1028F02B9
:1005000095029902CF02A402AA02AE02B402B80276
:10051000BC02C202C602CF02CA02D002D40280913B
:1005200080008F77809380000895809180008F7D78
:10053000F9CF80918000877FF5CF84B58F7784BD18
:10054000089584B58F7DFBCF8091B0008F77809325
:10055000B00008958091B0008F7DF9CF8091900018
:100560008F77809390000895809190008F7DF9CFD0
:1005700080919000877FF5CF8091A0008F77809346
:10058000A00008958091A0008F7DF9CF8091A000F8
:10059000877FF5CF809120018F7780932001089588
:1005A000809120018F7DF9CF80912001877FF5CF49
:1005B000CF93DF93282F30E0F901E254FE4F84916E
:1005C000F901E858FE4FD491F901EE5CFE4FC49159
:1005D000CC2399F0811185DFEC2FF0E0EE0FFF1FA7
:1005E000E85EFE4FA591B491EC91ED2381E090E09F
:1005F00009F480E0DF91CF91089580E090E0FACF98
:100600001F93CF93DF93282F30E0F901E254FE4F80
:100610008491F901E858FE4FD491F901EE5CFE4F48
:10062000C491CC23A1F0162F81115BDFEC2FF0E0F9
:10063000EE0FFF1FE250FF4FA591B4918FB7F894D2
:10064000EC91111108C0D095DE23DC938FBFDF91B0
:10065000CF911F910895DE2BF8CF0F931F93CF9367
:10066000082F082E000C110B20917E0A022E000C80
:10067000330B02171307B9F080937E0AC0E0809114
:10068000850AC81780F4EC2FF0E0B8010C2E02C0E8
:10069000759567950A94E2F76170E458F54F858186
:1006A000AFDFCF5FECCF8091880A882329F08130BB
:1006B00041F18FEF9FEF21C08091870A863308F0C8
:1006C000865320917B00982F9870277F922B9093D0
:1006D0007B008770806480937C0080917A008064C6
:1006E00080937A0080917A0086FDFCCF909178000B
:1006F00080917900892798278927CF911F910F91A1
:1007000008958091870ACF911F910F9151CFCF9378
:10071000DF9390E0FC01E858FE4F24918E5C9E4FE1
:10072000FC0184918823C9F090E0880F991FFC0197
:10073000EC51FF4FA591B491FC01E250FF4FC591E0
:10074000D49161110DC09FB7F8948C9120958223AC
:100750008C938881282328839FBFDF91CF910895B0
:10076000623051F49FB7F8943C91822F8095832397
:100770008C93E8812E2BEFCF8FB7F894EC912E2B32
:100780002C938FBFEACF3FB7F8948091C906909120
:10079000CA06A091CB06B091CC0626B5A89B05C091
:1007A0002F3F19F00196A11DB11D3FBFBA2FA92FF0
:1007B000982F8827BC01CD01620F711D811D911DED
:1007C00042E0660F771F881F991F4A95D1F7089559
:1007D0008F929F92AF92BF92CF92DF92EF92FF9251
:1007E0004B015C01D0DF6B017C01CDDF6C197D0911
:1007F0008E099F09683E734081059105B0F321E0A1
:10080000821A9108A108B10888EEC80E83E0D81EAC
:10081000E11CF11C81149104A104B10431F7FF9093
:10082000EF90DF90CF90BF90AF909F908F90089502
:100830002FB7F8946091C5067091C6068091C706DF
:100840009091C8062FBF0895FC01848187FD04C0E4
:1008500091E069276383D4DE80E00895FC01808500
:1008600080FD04C082FB882780F9089580E0089508
:10087000FC019085957081E0953009F080E0089545
:10088000862F642F44CFFC01818592DE21E0892BE5
:1008900009F420E0822F08950F931F93CF93DF93E5
:1008A0008BEF96E062DD892BA1F18BEF96E03BDDCB
:1008B0008C3329F41092C3061092C206F1CF8A300D
:1008C000B1F4C2E6D2E00EE516E089919991009765
:1008D00039F0F801208161E0213309F060E090DE19
:1008E0000F5F1F4FF2E0CA36DF0779F7E3CF2091A1
:1008F000C2063091C30624363105E4F6F901E25A06
:10090000F94F80832F5F3F4F3093C3062093C20679
:10091000C7CFDF91CF911F910F91089532DD8111E3
:10092000BBDF80E090E0892B49F080E090E0892BEC
:1009300029F00E94000081110E94000080E090E0F8
:10094000892B49F080E090E0892B29F00E9400007B
:1009500081110E94000080E090E0892B49F080E046
:1009600090E0892B29F00E94000081110C94000076
:100970000895DC01ED91FD918081ED91FD919081D3
:10098000ED91FD916C9163708E2309F064609F235B
:1009900009F06860E6EDF4E0E60FF11D65956595F8
:1009A0006D936D917D918D919D91099423C01AC095
:1009B00012C016C010C01EC009C014C013C006C0AB
:1009C00019C009C00DC007C00DC014C062507040EE
:1009D000804090400BC0615070408040904006C005
:1009E0006E5F01C06F5F7F4F8F4F9F4F9E938E93BF
:1009F0007E936E930895CF93DF93EC018B858230C5
:100A000058F4F894CE01B5DF6F81788589859A8591
:100A10007894DF91CF910895F894F6CF8F929F92BA
:100A2000AF92BF920F931F93CF93DF93CDB7DEB7F3
:100A3000A1970FB6F894DEBF0FBECDBF19A242300A
:100A400008F44AE08E010F5D1F4F842E912CB12CCB
:100A5000A12CA50194010E941E0FE62FB901CA0125
:100A6000EA303CF5E05DD801EE938D01232B242B79
:100A7000252B79F790E080E0109761F0FD0101905F
:100A80000020E9F73197AF014A1B5B0BBD018BEFEB
:100A900096E00DDCA1960FB6F894DEBF0FBECDBF79
:100AA000DF91CF911F910F91BF90AF909F908F904A
:100AB0000895E95CD8CF009761F0FC010190002017
:100AC000E9F73197AF01481B590BBC018BEF96E05A
:100AD000EECB90E080E00895AF92BF92DF92EF926C
:100AE000FF920F931F93CF93DF93EC01D62EF42E3A
:100AF000122F84E090E00E94640FFC01F0821183C9
:100B00000283E3828EE193E0998388838FEF8A8367
:100B10008B838C838A878B878C8784E089878F017E
:100B20005E0185E0A80EB11CF12CF80181918F01C6
:100B300087FD33C0F50181935F0161E0E8DDF39447
:100B4000F4E0FF12F2CF8FEF8C8384E293E099837D
:100B500088838B8587FD0FC0282F082E000C330B50
:100B6000D216130641F09A85913011F460E048DD09
:100B700060E08B85CCDD82E08A87DB8662E08D2DAC
:100B8000C6DD81E08C87DF91CF911F910F91FF909F
:100B9000EF90DF90BF90AF900895F986D4CFCF93B8
:100BA000DF93EC0188819981009711F00E94001079
:100BB000198218821D821C821B821A82DF91CF91BA
:100BC0000895FC0180819181009711F00C94001030
:100BD00008950E9465110F931F93CF93DF93EC014B
:100BE00088819981009759F02A813B812617370720
:100BF00030F081E0DF91CF911F910F9108958B012B
:100C00006F5F7F4F0E948910009759F09983888306
:100C10001B830A832C813D81232B59F7FC01108211
:100C2000E8CF80E0E7CFEF92FF920F931F93CF932F
:100C3000DF93EC017B018A01BA01CDDF81110AC08B
:100C4000CE01ADDFCE01DF91CF911F910F91FF90CB
:100C5000EF9008951D830C83B701888199810E94CC
:100C60007A11F0CF1F920F920FB60F9211240BB68C
:100C70000F922F933F934F935F936F937F938F9335
:100C80009F93AF93BF93EF93FF938BEF96E082DB3D
:100C9000FF91EF91BF91AF919F918F917F916F9154
:100CA0005F914F913F912F910F900BBE0F900FBE10
:100CB0000F901F9018951F920F920FB60F9211244C
:100CC0000BB60F922F938F939F93EF93FF93E09127
:100CD0000B07F0910C078081E0911107F09112074A
:100CE00082FD1DC09081809114078F5F8F732091CA
:100CF0001507821741F0E0911407F0E0E550F94F35
:100D0000958F80931407FF91EF919F918F912F9171
:100D10000F900BBE0F900FBE0F901F901895808103
:100D2000F2CF1F920F920FB60F9211242F933F9381
:100D30008F939F93AF93BF938091C5069091C60602
:100D4000A091C706B091C8063091C40623E0230FD6
:100D50002D3758F50196A11DB11D2093C40680932F
:100D6000C5069093C606A093C706B093C8068091A7
:100D7000C9069091CA06A091CB06B091CC06019607
:100D8000A11DB11D8093C9069093CA06A093CB06FE
:100D9000B093CC06BF91AF919F918F913F912F91CE
:100DA0000F900FBE0F901F90189526E8230F029604
:100DB000A11DB11DD2CF1F920F920FB60F92112419
:100DC0000BB60F922F933F934F935F936F937F9345
:100DD0008F939F93AF93BF93EF93FF9380915406AC
:100DE00090915506C6DDFF91EF91BF91AF919F9114
:100DF0008F917F916F915F914F913F912F910F90C4
:100E00000BBE0F900FBE0F901F9018951F920F9260
:100E10000FB60F9211240BB60F922F933F934F935F
:100E20005F936F937F938F939F93AF93BF93EF9352
:100E3000FF9380915206909153069BDDFF91EF91B5
:100E4000BF91AF919F918F917F916F915F914F91E2
:100E50003F912F910F900BBE0F900FBE0F901F90E0
:100E600018951F920F920FB60F9211240BB60F9286
:100E70002F933F934F935F936F937F938F939F93A2
:100E8000AF93BF93EF93FF9380915C0690915D06C3
:100E900070DDFF91EF91BF91AF919F918F917F9105
:100EA0006F915F914F913F912F910F900BBE0F90DB
:100EB0000FBE0F901F9018951F920F920FB60F92B2
:100EC00011240BB60F922F933F934F935F936F9321
:100ED0007F938F939F93AF93BF93EF93FF938091F3
:100EE0005A0690915B0645DDFF91EF91BF91AF915E
:100EF0009F918F917F916F915F914F913F912F9132
:100F00000F900BBE0F900FBE0F901F9018951F9261
:100F10000F920FB60F9211240BB60F922F933F939F
:100F20004F935F936F937F938F939F93AF93BF93F1
:100F3000EF93FF9380915806909159061ADDFF9127
:100F4000EF91BF91AF919F918F917F916F915F9141
:100F50004F913F912F910F900BBE0F900FBE0F90AE
:100F60001F9018951F920F920FB60F9211240BB677
:100F70000F922F933F934F935F936F937F938F9332
:100F80009F93AF93BF93EF93FF93809156069091F9
:100F90005706EFDCFF91EF91BF91AF919F918F9139
:100FA0007F916F915F914F913F912F910F900BBE69
:100FB0000F900FBE0F901F90189590E0823090F424
:100FC00004968330910569F17CF481309105C9F074
:100FD0000297F9F0809169008C7F816080936900AD
:100FE000E89A08950297EDCF8430910511F10597A5
:100FF00089F780916A00837F846080936A00ED9A0C
:10100000089580916900837F846080936900E99AE4
:101010000895809169008F7C806180936900EA9ACD
:101020000895809169008F73806480936900EB9AC2
:10103000089580916A008C7F816080936A00EC9AA9
:101040000895823161F130F4823079F08330A9F073
:1010500080E008958431B9F0E0F08531C9F77093EC
:1010600057066093560682E005C07093530660935E
:10107000520680E0A2DF81E00895709355066093E8
:10108000540681E0F7CF709359066093580683E0C9
:10109000F1CF70935B0660935A0684E0EBCF7093B8
:1010A0005D0660935C0685E0E5CF0F931F93CF93B9
:1010B000DF93EC01062F142F62E0802F28DB62E023
:1010C000812F25DB802F90E0FC01EE5CFE4FE49148
:1010D000F0E0EE0FFF1FE85EFE4FA591B491B983DB
:1010E000A883FC01E858FE4F24912C83812F90E0C7
:1010F000FC01EE5CFE4FE491F0E0EE0FFF1FE85EB6
:10110000FE4F459154915B834A83FC01E858FE4FA2
:10111000E491ED831F82188619861A868BE39FE17E
:101120000197F1F78C91282391E009F490E0DA011E
:101130008C91E82309F092609E83BE01802F81DFAD
:101140008B87BE01812F7DDF9B85890F8B87DF9188
:10115000CF911F910F910895EF920F931092FE0679
:101160001092FD0688EE93E0A0E0B0E08093FF06C9
:1011700090930007A0930107B09302078AE293E0DF
:101180009093FC068093FB0685EC90E09093080713
:101190008093070784EC90E090930A0780930907F7
:1011A00080EC90E090930C0780930B0781EC90E02B
:1011B00090930E0780930D0782EC90E090931007B8
:1011C00080930F0786EC90E09093120780931107AD
:1011D0001092140710921507109216071092170715
:1011E000A8E9B7E090E080E041E2FC013E9621E012
:1011F00030E08630910510F430E020E0E20FF31F7C
:1012000040935700E491ED9301968930910569F779
:1012100087E1E82E09E12BE14DE166E18CE79AE0F8
:101220005BDC97E6E92E06E625E644E663E68FE614
:101230009AE052DC42E063E08FE09AE036DF80E43F
:1012400093E090931C0A80931B0A8BE493E09093A5
:101250001E0A80931D0A46E065E08FE19AE025DFD3
:1012600086E593E090932C0A80932B0A81E693E025
:1012700090932E0A80932D0A43E361E28FE29AE075
:1012800014DF8CE693E090933C0A80933B0A87E757
:1012900093E090933E0A80933D0A49E26FE28FE328
:1012A0009AE003DF82E893E090934C0A80934B0A24
:1012B0008FE893E090934E0A80934D0A48E16FE3E4
:1012C0008FE49AE0F2DE8CE993E090935C0A8093DD
:1012D0005B0A8DEA93E090935E0A80935D0A41E495
:1012E0006AE18FE59AE0E1DE8EEB93E090936C0A81
:1012F00080936B0A8FEC93E090936E0A80936D0A53
:10130000E7EAF7E02CE333E08AE090E031832083E2
:101310001282138214821582978386831086118627
:101320003E964AE0EF30F40789F71092A207109238
:10133000A1071092A4071092A3071092A60710927B
:10134000A50750E040E061E174E081EA97E00F9189
:10135000EF9069CCCF93DF93CDB7DEB767970FB629
:10136000F894DEBF0FBECDBF789484B5826084BD93
:1013700084B5816084BD85B5826085BD85B5816099
:1013800085BD80916E00816080936E001092810017
:1013900080918100826080938100809181008160D2
:1013A0008093810080918000816080938000809193
:1013B000B10084608093B1008091B000816080931F
:1013C000B0008091910082608093910080919100A3
:1013D0008160809391008091900081608093900063
:1013E0008091A10082608093A1008091A100816022
:1013F0008093A1008091A00081608093A0008091E3
:10140000210182608093210180912101816080937C
:1014100021018091200181608093200180917A00D8
:10142000846080937A0080917A00826080937A0051
:1014300080917A00816080937A0080917A00806840
:1014400080937A001092C10009E9C02E07E0D02EE7
:101450008E010F5F1F4FD6018D916D011B861A867D
:101460001D861C861F861E8640E1B80190E0BDD413
:10147000F80101900020E9F73197AF01401B510BB3
:10148000B801CE010A96CFDB1A8219821C821B8218
:101490001E821D826091A1077091A20761157105DE
:1014A00031F04091A5075091A607C801BCDB8E859D
:1014B0009F85AA84BB84ED80FE80E80EF91EA114EE
:1014C000B10409F439C0892B79F0B701C80183DB75
:1014D000882391F129813A818D819E81B501820F06
:1014E000931F08D7FE82ED8269817A8161157105AB
:1014F00031F14D815E8181EA97E095DBC80161DBC6
:10150000CE010A965EDBB1EACB16B7E0DB0609F046
:10151000A2CF0091A1071091A2070115110599F022
:10152000F8018081882379F0082E000C990BD1D620
:10153000D8018D938D01F4CFC80131DBD5CF81EA7D
:1015400097E02DDBDBCF1DECE12E16E0F12E10E055
:10155000812F83D8F70181937F011F5F1031C1F77D
:1015600007EA17E0AAE6EA2EA2E0FA2EBAE0AB2ECE
:10157000B12CD701DC9011967C91D801ED91FC91B2
:101580000280F381E02D42E050E06D2DC8011995F5
:10159000F801D18610860190F081E02D0190F08154
:1015A000E02DC8011995882339F0D80118968C913F
:1015B0001897836018968C933BD9F80162837383E4
:1015C00084839583B782A682F4E0EF0EF11C025F5C
:1015D0001F4F2AE00F30120761F6EBEFCE2EE6E048
:1015E000DE2E03EE16E0FFE0EF2EFAE0FF2EC7013D
:1015F00002DAD8016D937D938D939D938D01B0E1B7
:10160000EB0EF11CC016D10691F762E6E62E62E001
:10161000F62E7AE6A72E72E0B72E8701F801C19068
:10162000D1908F01C114D10439F061E08C2D6FD8B5
:1016300061E08C2D0E940003A016B10679F768E8DE
:1016400073E180E090E0C4D8D7018D919D917D0138
:10165000009719F060E00E940003E016F106A1F780
:1016600080EE93E0805F934039F461E08CE04FD8E6
:1016700061E08CE00E94000368EE73E080E090E09F
:10168000A7D8E0910B07F0910C0782E08083E091EE
:101690000707F09108071082E0910907F0910A0707
:1016A00080E1808310921307E0910F07F0911007FB
:1016B00086E08083E0910D07F0910E0780818061C4
:1016C0008083E0910D07F0910E0780818860808310
:1016D000E0910D07F0910E07808180688083E09192
:1016E0000D07F0910E0780818F7D808382E390E06B
:1016F000A0E0B0E08093FF0690930007A09301075D
:10170000B093020722242394312C92D82B013C0160
:101710008091180290911902A0911A02B0911B02B7
:10172000AC01BD014854544F6F4F7F4F44165506CE
:101730006606770630F4481659066A067B0608F0F6
:101740003CC085E392E00E94380280EE93E0B3D97A
:1017500083E392E00E9438024AE065E070E080E0B6
:1017600090E05CD981E392E00E94380282E192E04D
:10177000A2D98FE292E00E9438024091A5075091D1
:10178000A6076091A1077091A2078BEF96E00E94D7
:1017900057018DE292E00E94380240921802509266
:1017A000190260921A0270921B0240920E0250922D
:1017B0000F02609210027092110243EEC42E46E0B6
:1017C000D42E0FE01AE0F12CE12CE1E0E88B20EEC2
:1017D00033E02F5F334009F0188AD8011C968D91B1
:1017E0009C91B3E08B349B0709F438C18C5693402D
:1017F00009F434C1D8011E962D913C9181E0B3E0EB
:1018000020343B0721F02757334009F080E0A888B7
:10181000AA2009F425C1882309F422C1C801EBD804
:1018200024E030E040E050E02BD349015A01F601BA
:1018300080819181A281B38188159905AA05BB0594
:101840000CF016C181E02091E1063091E2062130D2
:10185000310509F080E0F8898F2341F080914D0A2D
:1018600090914E0A21E0E216F10421F0D8011E9673
:101870008D919C9120D98BE292E00E943802409297
:101880000E0250920F026092100270921102F60145
:1018900081929192A192B1926F01FFEFEF1AFF0A2C
:1018A000005F1F4F26E0E216F10409F08ECF2AE612
:1018B000822E22E0922E07EA17E01E8A1D8A30EE61
:1018C000E32E33E0F32ED80118968C9118978B7F76
:1018D00018968C931897ED91FC910190F081E02D72
:1018E000C80119958F8BF801808586958170AF8826
:1018F000A81609F4DFC00E941804D80112966D934F
:101900007D938D939C93159718968C91B2E08B27BD
:10191000F8018087C8010E942E04811106C0C80109
:101920000E943804882309F487C0F401C080D18064
:10193000C6018B7F8397C9F1FBE2CF16D104A9F1D1
:101940002DE2C216D10489F132E1E31634E0F30648
:1019500009F4ECC048E2E41644E0F40609F4E6C0F9
:101960005EE3E51654E0F50609F4E0C083E5E81609
:1019700084E0F80609F4DAC081E099E6E91694E01B
:10198000F90609F080E096012351310991E02330F6
:10199000310528F0ACE1CA16D10409F090E08823A3
:1019A00009F4C6C0992309F4C3C040920A025092B8
:1019B0000B0260920C0270920D021092E0061092DF
:1019C000DF06D40112968D919C9175D8C8010E94B2
:1019D0002E04882309F4D5C185E292E00E943802E2
:1019E000BBE2CB16D104D1F4A888AA20B9F080912B
:1019F000E1069091E206009709F0BAC13092E20642
:101A00002092E1064092000250920102609202028E
:101A10007092030261E080E00E94000364E670E0DF
:101A200080E090E00E94E80340920E0250920F0284
:101A300060921002709211022D893E892F5F3F4FF4
:101A40003E8B2D8B025F1F4F34E0830E911C4D891E
:101A50005E894C32510509F036CFC9C081E0D7CE3E
:101A6000C8010E94FB0422E030E040E050E0DCCE00
:101A700088169906AA06BB060CF009CF81E02091D2
:101A8000E1063091E2062130310509F080E0B889A5
:101A90008B2341F080914B0A90914C0AE1E0EE16C5
:101AA000F10421F0D8011C968D919C9104D889E213
:101AB00092E0E3CE0E941804D8011296AD90BD903A
:101AC000CD90DC9015979B01AC012A193B094C097C
:101AD0005D0916968D919C91B0E0A0E0281739071A
:101AE0004A075B0708F416CFD80118968C918170CD
:101AF000AF88A81609F40ECF0E941804D8011296D8
:101B00006D937D938D939C93159718968C91B1E06E
:101B10008B278460F80180870E941804D8011A96E8
:101B20006D937D938D939C931D97F4CE81E02BCF85
:101B3000B5E2CB16D10431F1E2E1EE16E4E0FE06A7
:101B400009F414C1F8E2EF16F4E0FF0609F40EC13F
:101B50002EE3E21624E0F20609F408C181E033E541
:101B6000E31634E0F30631F049E6E41644E0F40607
:101B700009F080E05AE1C516D10409F022CF88238C
:101B800009F41FCF80910A0290910B02A0910C02E0
:101B9000B0910D0283589F4FAF4FBF4F4816590663
:101BA0006A067B0620F13092E0062092DF06AD88BF
:101BB000BE88B092DE06A092DD06409206025092E8
:101BC00007026092080270920902C8010E942E0466
:101BD000882321F01092050210920402C8010E948D
:101BE0003804882321F0309205022092040280EE0E
:101BF00093E08F5F934001F5809100029091010284
:101C0000A0910202B091030288539D4CAF4FBF4F89
:101C100084159505A605B70520F41092E2061092EA
:101C2000E1068091E1069091E20660E0892B09F0DF
:101C300061E080E00E94000302E212E09DECE92EE8
:101C400096E0F92EB12C8B2D0E942D03D7019D918A
:101C50007D018917B1F0FD01319780838111A2C008
:101C6000F801C280D3806FE774E0C6014AD3892BA4
:101C700009F492C0C6010E945B058CE192E00E94CB
:101C80003802B3940C5F1F4FB0E1BB12DCCF8091E0
:101C90000E0290910F02A0911002B0911102AC01BE
:101CA000BD014C595F4F6F4F7F4F44165506660676
:101CB000770628F4481659066A067B0660F48CE01D
:101CC00092E00E94380240920E0250920F026092FF
:101CD0001002709211028091060290910702A09169
:101CE0000802B091090283589F4FAF4FBF4F841530
:101CF0009505A605B705B8F58091DF069091E00639
:101D0000019789F5E091DD06F091DE06EE0FFF1FE9
:101D1000EE0FFF1FE659FD4F828193810E945B0504
:101D20008091040290910502009709F054C088E068
:101D300092E00E94380264E670E080E090E00E9449
:101D4000E80340920E0250920F02609210027092CD
:101D500011021092E0061092DF06E9E0F0E0F09345
:101D60000502E09304020E948E04CFCC81E002CFF2
:101D7000019709F053CE1092E2061092E10660E05E
:101D80004ACEC8010E943804882309F447CE81E274
:101D900092E00E94380242CEC6010E945B0588E1B3
:101DA00092E06DCF813009F06CCFD8011296CD90C2
:101DB000DC906FE774E0C601A4D2892B31F0C60134
:101DC0000E945B0582E192E05ACFC6010E945B054A
:101DD0008EE092E054CF019709F0ADCF84E092E01D
:101DE000A8CF81EA97E00C94E105BB27FB015527BA
:101DF000AA27880F991FAA1FA41710F0A41B839568
:101E00005051B9F7A05DAA3308F0A95DA1930097DE
:101E100079F7B111B1931192CB0100C0DC01FC0143
:101E2000672F71917723E1F7329704C07C916D930E
:101E300070836291AE17BF07C8F30895A1E21A2E0E
:101E4000AA1BBB1BFD010DC0AA1FBB1FEE1FFF1F5E
:101E5000A217B307E407F50720F0A21BB30BE40BAE
:101E6000F50B661F771F881F991F1A9469F76095F5
:101E70007095809590959B01AC01BD01CF010895AF
:101E8000052E97FB16F400940FD057FD05D0D6DF32
:101E900007FC02D046F408C0509540953095219536
:101EA0003F4F4F4F5F4F0895909580957095619586
:101EB0007F4F8F4F9F4F0895EE0FFF1F881F8BBFDF
:101EC0000790F691E02D19940F931F93CF93DF9312
:101ED0008230910510F482E090E0E0918B0AF0915D
:101EE0008C0A30E020E0B0E0A0E0309799F42115B2
:101EF000310509F44AC0281B390B24303105D8F5C7
:101F00008A819B816115710589F1FB01938382832D
:101F1000FE0111C040815181028113814817590788
:101F2000E0F04817590799F4109761F012960C9356
:101F3000129713961C933296CF01DF91CF911F9188
:101F40000F91089500938B0A10938C0AF4CF2115FA
:101F5000310551F04217530738F0A901DB019A010E
:101F6000BD01DF01F801C1CFEF01F9CF90938C0AD9
:101F700080938B0ACDCFFE01E20FF31F81939193E3
:101F80002250310939832883D7CF2091890A309193
:101F90008A0A232B41F420911E0230911F023093B4
:101FA0008A0A2093890A20911C0230911D02211572
:101FB000310541F42DB73EB74091200250912102E6
:101FC000241B350BE091890AF0918A0AE217F30786
:101FD000A0F42E1B3F0B2817390778F0AC014E5F99
:101FE0005F4F2417350748F04E0F5F1F50938A0A42
:101FF0004093890A819391939FCFF0E0E0E09CCFDA
:10200000CF93DF930097E9F0FC013297138212829D
:10201000A0918B0AB0918C0AED0130E020E010977E
:10202000A1F420813181820F931F2091890A309180
:102030008A0A2817390709F061C0F0938A0AE093E9
:10204000890ADF91CF910895EA01CE17DF07E8F5FD
:102050004A815B819E0141155105B1F7E901FB837E
:10206000EA8349915991C40FD51FEC17FD0761F41C
:10207000808191810296840F951FE901998388835D
:10208000828193819B838A83F0E0E0E012968D91B8
:102090009C9113970097B9F52D913C911197CD0123
:1020A0000296820F931F2091890A30918A0A28177D
:1020B000390739F6309751F510928C0A10928B0A35
:1020C000B0938A0AA093890ABCCFD383C28340818C
:1020D0005181840F951FC817D90761F44E5F5F4F78
:1020E00088819981480F591F518340838A819B8140
:1020F000938382832115310509F0B0CFF0938C0AC8
:10210000E0938B0A9ECFFD01DC01C0CF13821282C7
:10211000D7CF4F925F926F927F928F929F92AF92A2
:10212000BF92CF92DF92EF92FF920F931F93CF93C4
:10213000DF938C01009791F4CB01DF91CF911F9138
:102140000F91FF90EF90DF90CF90BF90AF909F9056
:102150008F907F906F905F904F90B6CEFC01E60F0E
:10216000F71F9C0122503109E217F30708F4AAC0B7
:10217000D901CD91DC911197C617D70718F1C53059
:10218000D10570F0CE0104978617970748F0C61B5B
:10219000D70B2297C193D1936D937C93CF0130DFFE
:1021A000C801DF91CF911F910F91FF90EF90DF90C9
:1021B000CF90BF90AF909F908F907F906F905F90E7
:1021C0004F9008955B01AC1ABD0A4C018C0E9D1E08
:1021D000A0918B0AB0918C0A512C412CF12CE12C4E
:1021E000109731F58091890A90918A0A881599058E
:1021F00009F05CC04616570608F058C080911C02D2
:1022000090911D02009741F48DB79EB74091200236
:1022100050912102841B950BE817F90708F052C072
:10222000F0938A0AE093890AF90171836083B8CF39
:102230008D919C91119712966C90129713967C90A9
:102240001397A815B90559F56C0142E0C40ED11CCD
:10225000CA14DB0420F1AC014A195B09DA011296B9
:10226000159780F06282738251834083D9016D9308
:102270007C93E114F10471F0D7011396FC93EE9373
:1022800012978ECF22968C0F9D1FF9019183808328
:10229000F301EFCFF0938C0AE0938B0A81CF4816BD
:1022A000590608F42C017D01D3019ACFCB010CDE35
:1022B0007C01009739F0AE01B80113D0C801A0DE4F
:1022C00087016ECF10E000E06BCF81E090E0F894E2
:1022D00032C09111089581568A5108F48052855870
:1022E0000895FB01DC0102C001900D924150504065
:1022F000D8F70895FB01DC0101900D920020E1F771
:102300000895FB0151915523A9F0BF01DC014D91C6
:1023100045174111E1F759F4CD010190002049F032
:102320004D9140154111C9F3FB014111EFCF81E0FF
:1023300090E00197089511E0C4E2D1E000E005C00B
:10234000802FFE01B9DD2196011DC532D10780E045
:082350000807B1F7F894FFCF74
:10235800FFFFFFFF0900FFFFFFFFFFFFFFFFFFFF7A
:10236800FFFF332E312E3500FFFFFFFF00008D0ADF
:102378008000000083040100890402008F04030028
:10238800950404009B040500A1040600A7040700A7
:10239800AD040800B3040900B9040A00BF040B0027
:1023A800C5040C00CB040D00D1040E00D7040F00A7
:1023B800DD040F001100130015003500E3040400CC
:1023C800F0040700FD0408000A05090012050A00C8
:1023D8001D050B0025050C002D050D0036050E000A
:1023E8003F051000480512005005140058051E004E
:1023F80061051F00670520006F0522007505230091
:102408007B052400860525008C05260099052700F4
:102418009F052800AC052A00B2052B00B8052C0042
:10242800C3052D00C9052E00D7053000DF05320091
:10243800E5053400EB053600F4053700FA053800E9
:102448000006390006063A000C063B0012063C005E
:1024580018063E001E0640002806420035064300C6
:102468003B06440041064500470600000000E90518
:1024780000000000240400000000EC015701840162
:102488005202B5019301A701000000004304400473
:10249800454E435F4844475F444E00454E435F48BE
:1024A80044475F555000454E435F4352535F555074
:1024B80000454E435F4352535F444E00454E435FD1
:1024C800414C545F555000454E435F414C545F4466
:1024D8004E00454E435F52414E47455F444E0045CE
:1024E8004E435F52414E47455F555000454E435F4E
:1024F800464D535F494E4E45525F555000454E4339
:102508005F464D535F494E4E45525F444E00454E1F
:10251800435F464D535F4F555445525F444E004507
:102528004E435F464D535F4F555445525F555000DB
:102538005265616C53696D476561722D474355005B
:102548005265616C53696D476561722D473500525C
:1025580065616C53696D476561722D474643353037
:1025680030005265616C53696D476561722D473162
:1025780030303050464431005265616C53696D47C4
:102588006561722D47313030304D46443100526517
:10259800616C53696D476561722D47313030305831
:1025A8004644005265616C53696D476561722D47F9
:1025B8003130303058464431005265616C53696D92
:1025C800476561722D473130303058464432002E0D
:1025D80053570042544E5F5A0042544E5F430042E4
:1025E800544E5F490042544E5F4E0042544E5F5471
:1025F8000042544E5F590042544E5F420042544ECE
:102608005F480042544E5F4D0042544E5F530042B3
:10261800544E5F580042544E5F410042544E5F474B
:102628000042544E5F4C0042544E5F520042544E9A
:102638005F570042544E5F414C545F53594E43001C
:1026480042544E5F4844475F53594E430042544EEC
:102658005F4352535F53594E430042544E5F454EB9
:10266800540042544E5F4449524543540042544E2C
:102678005F46504C0042544E5F434C520042544E09
:102688005F4D454E550042544E5F50524F430042F5
:10269800544E5F464C49500042544E5F464D5300DD
:1026A80042544E5F434F4D0042544E5F585044527F
:1026B8000042544E5F440042544E5F4E4156004221
:1026C800544E5F4A0042544E5F4F0042544E5F5092
:1026D800414E5F55500042544E5F550042544E5F84
:1026E80050414E5F53594E430042544E5F4500429D
:1026F800544E5F50414E5F4C4546540042544E5F25
:102708004B0042544E5F500042544E5F50414E5F62
:10271800444E0042544E5F560042544E5F50414E64
:102728005F52494748540042544E5F535043004259
:10273800544E5F460042544E5F510042544E5F4231
:102748004B53500042544E5F320042544E5F3500A6
:1027580042544E5F380042544E5F300042544E5F40
:10276800330042544E5F360042544E5F39004254A3
:102778004E5F4D494E55530042544E5F464D535F90
:1027880053594E430042544E5F310042544E5F3419
:102798000042544E5F370042544E5F504552494FF5
:0227A8004400EB
:00000001FF
